:03000000024201B8
:0C42010078FFE4F6D8FD75817202424897
:10240A0020000A3C2E2E2E3E004950436F6E6E6508
:10241A0063745245510A004950436F6E6E65637486
:10242A00000A49504E6F41434B210A003E432C5645
:10243A002C43432CC0E4E0EFF2E5F020D1E8EDEACA
:10244A00EEEC49500A003E432C4D41432C253032D4
:10245A0062583A25303262583A25303262583A2563
:10246A00303262583A25303262583A253032625850
:10247A002C4D414320E0E4F0E5F10A003E432C569E
:10248A0045522C20332E3220EEF22025732025735C
:10249A002CC2E5F0F1E8FF20495020ECEEE4F3EB22
:1024AA00FF0A00466562203231203230303900316D
:1024BA00303A33383A3030003E432C4C442C505298
:1024CA004F473A2020202020202020202020202092
:1024DA0020202020202020202020202020202020F2
:1024EA0020202020202020202020202020202020E2
:1024FA0020202020202020202020202020202020D2
:10250A0020202020202020202CC4E0F2E020EFF020
:10251A00EEF8E8E2EAE828F4E0E9EB290A003E2AC4
:10252A002C312CCEF1EDEEE2EDFBE520EFE0F0E010
:10253A00ECE5F2F0FB20F1E5F2E5E2EEE3EE20E86D
:10254A00EDF2E5F0F4E5E9F1E00A003E412C413014
:10255A00312C2562752E2562752E2562752E25620F
:10256A00752C495020E0E4F0E5F120E0E4E0EFF2D8
:10257A00E5F0E00A003E412C4130322C2562752EEE
:10258A002562752E2562752E2562752C495020E02C
:10259A00E4F0E5F120EEF1ED2E20F1E5F0E2E5F0D0
:1025AA00E00A003E412C4130332C2562752E25620B
:1025BA00752E2562752E2562752C495020E0E4F0AF
:1025CA00E5F120F0E5E72E20F1E5F0E2E5F0E00A9A
:1025DA00003E412C4130342C2562752E2562752E21
:1025EA002562752E2562752CCCE0F1EAE020F1E532
:1025FA00F2E80A003E412C4130352C2562752E2521
:10260A0062752E2562752E2562752CD8EBFEE70AB7
:10261A00003E2A2C312CC4EEEF2E20EFE0F0E0EC45
:10262A00E5F2F0FB20F1E5F2E5E2EEE3EE20E8ED7B
:10263A00F2E5F0F4E5E9F1E00A003E422C533031CC
:10264A002C2562752CC6E4E0F2FC20E7E0EFF0EE00
:10265A00F1E020F1EEE5E4E8EDE5EDE8FF20EEF249
:10266A0020F1E5F0E2E5F0E00A003E422C53303278
:10267A002C2562752CCEE1ECE5ED20F120F1E5F098
:10268A00E2E5F0EEEC20E1E5E720EAE2E8F2E0ED4F
:10269A00F6E8E90A003E422C5330332C2562752CA9
:1026AA00CFE5F0E5E7E0EFF3F1EA20EFF0E820EF1D
:1026BA00EEF2E5F0E520F1E2FFE7E820F120F1E5AE
:1026CA00F0E2E5F0EEEC0A003E454E440A000A4408
:1026DA00756D705820202020203030203031203075
:1026EA003220303320303420303520303620303715
:1026FA0020303820303920304120304220304320E9
:10270A003044203045203046000A3A003A20000A78
:10271A00000A44756D70442020202020303020307B
:10272A0031203032203033203034203035203036DA
:10273A0020303720303820303920304120304220B4
:10274A003043203044203045203046004572722004
:10275A006B657900526420656570726F6D0A00526C
:10276A0064204D454D0A00526420436F64650A0097
:10277A00577269746520436F64650A00446562751F
:10278A00674950204F4E0A004465627567495020D8
:10279A004F46460A00446562756755736572204F55
:1027AA006E0A00446562756755736572204F464626
:1027BA000A0044656275674D7367204F6E0A0044CC
:1027CA00656275674D7367204F46460A00436F6E10
:1027DA00666967206C6F636B210A00577220656512
:1027EA0070726F6D0A00205361766520656570729C
:1027FA006F6D210A00457272204D414321004C6FD2
:10280A0061643E3E002A003C4130313D003C41308B
:10281A00323D003C4130333D003C4130343D003CC8
:10282A004130353D003C21003C5330313D003C53A2
:10283A0030323D003C5330333D003C5330353D008F
:06284A003C5330363D0056
:064B0100010B0001090098
:104AF100C28E438910758BFF758DB7D2ABD28E22D2
:03001B000241712E
:10417100C0E0C083C082C0D0C28E758BFF758DB781
:1041810020060675A61E75A6E10509D202E50B609B
:1041910002050BE50AD394014002150A050EE50E4E
:1041A100540F7048D20EE50E543F7012D200906643
:1041B1008BE0600A04F0E0D394B44002D20690662A
:1041C10086E0600204F0906104E0600214F0906601
:1041D1008CE0D394014003E014F0300502050CE5B6
:1041E1000DD394644004D2068002050DE508D394F2
:1041F1000140021508D28ED0D0D082D083D0E032D7
:1018BB00C291C290D2B5C20B7D027C007F07124A47
:1018CB00BA8F54E554646060097D017F60124A351C
:1018DB00D20BE4FDFC7F0B124ABA8F54E55430E671
:1018EB00097D04E4FF124A59D20B7D017C007F076E
:1018FB00124ABA8F54E5547008FD7FFF124A35D255
:10190B000B300B03126000C288C2A8C2AA758900F3
:10191B001245A990633EE0B4FA06A3E064CE607B67
:10192B00E4F55474362554F582E43463F583E4F01E
:10193B000554E554B443EC90633E74FAF0A374CEB3
:10194B00F0A374CCF0906344740AF0E4A3F0A30406
:10195B00F0A3F090633A74FFF0A3F0A3F0E4A3F0CC
:10196B00906355740AF0E4F554E5542401FFE43315
:10197B00FE74362554F582E43463F583E0FD124A98
:10198B00110554E554C3944340DFE4F5A775A61E37
:10199B0075A6E1907FF0F0A3F080FE90634974038D
:1019AB00F0A374CCF0E4906348F0123EC7C2B512BA
:1019BB004041C20612489AD20BC20DC20C906576FA
:1019CB007408F09062B47424F0E4A3F090633EE0EA
:1019DB009062B6F090633FE09062B7F0906340E0A6
:1019EB009062B8F0906341E09062B9F0906342E08E
:1019FB009062BAF0906343E09062BBF0750A01E429
:101A0B00906577F0C207C208C209C20A200B18AF53
:101A1B0054FE7D03123D0BE4FF123F917E247F0A9F
:101A2B00E4FBFDFC123A1890668BE060037401F046
:101A3B00E4906104F0F50C906575F0F50D124AF128
:101A4B0075A70775A61E75A6E1D2AFE4F50D9061DB
:101A5B0004E0700312112490668CE06401701D90F9
:101A6B0080007410F09080A874FFF0A3F0A3F0A393
:101A7B00F0E490668CF0D20BC20CC20D908008E0A3
:101A8B00F55430E405D2077410F0E55430E508D274
:101A9B00099080087420F0E55430E608D208908055
:101AAB00087440F0E50CC394034019908002E4F0F5
:101ABB00908001F0908000F0E50C94064006E4F570
:101ACB000C12489A9080A0E070031247139080B8D4
:101ADB00E070031246279080D0E0700312483E90CE
:101AEB008000E07013300710123B1F906331EFF052
:101AFB00D3940040031208E1908002E070069080BE
:101B0B0000E06005D205021A56C205E4F50C90619F
:101B1B0004E06003021A56200B12906578E0600C0B
:101B2B007E247F0C123C23E4906578F0300912126E
:101B3B003675906331EFF0D394004005E0FF12004F
:101B4B0022200803021CCC123379906331EFF07022
:101B5B0003021A56906375E054BF247F7003021C76
:101B6B0035147003021C0D24026003021C6E200B43
:101B7B00077E247F13123C23200F03021CCC90639F
:101B8B004DE07006906351E06067906682E0FF90D5
:101B9B00634DE0B50724906683E0FE90634EE0B59D
:101BAB000618906684E0FE90634FE0B5060C9066D5
:101BBB0085E0FE906350E06E6037906351E06F609C
:101BCB0003021CCC906683E0FF906352E06F6003CE
:101BDB00021CCC906684E0FF906353E06F600302BD
:101BEB001CCC906685E0FF906354E06F6003021C91
:101BFB00CCC2039065777401F0124B0A750A01028F
:101C0B001CCC90668BE060037401F090667AE0FF69
:101C1B00906377E06F6003021CCC90667AE004F06F
:101C2B00E4F50A906575F0021CCC300303021CCC62
:101C3B00906344E07003021A56906355740AF012D5
:101C4B004B09D203E4F50A906575F090668604F0B3
:101C5B00E4906679F0A3F0200B677E247F21123C81
:101C6B0023805E90668BE060037401F0300352902A
:101C7B006375E020E74B906377E0FF906679E0FEB9
:101C8B006F600D906681E07007EE146F70338013F8
:101C9B00906679E004F0906331E0FFD39404400345
:101CAB00124A7D9060007482F0A37401F090637708
:101CBB00E0906002F07E607F007D03124314021AF5
:101CCB0056200303021DE4E50A70681237E6EF6045
:101CDB00237E647F75906476E02404FD1243149098
:101CEB006681E07009906355E0F50A021A56E4F537
:101CFB000A021A56906686E0D3943C403690668171
:101D0B00E0703090668604F0124B08E4906475F036
:101D1B00A37412F090667AE0906477F0A374FDF0F0
:101D2B0090610563A20190647963A2017F12122F67
:101D3B002D809E12001E8F54E554B4011590600047
:101D4B007483F0E4A3F07E607F007D0212431402E3
:101D5B001A56E554D39401401C9060007483F0A391
:101D6B007401F0E55424FEA3F07E607F007D031226
:101D7B004314021A56E50A64016003021A56906571
:101D8B0075E004F0200B077E247F2B123C2390631D
:101D9B0055E0C394C85004E02432F0906575E0C35D
:101DAB009405400DC203E4906577F0124B0A021ABA
:101DBB00567C667D82906349E0FAA3E0FB7F0212BA
:101DCB0044A57E647F75906476E02404FD12431471
:101DDB00906355E0F50A021A56E50A6401600302A6
:101DEB001A56906577E014604624FE604214700327
:101DFB00021ED724046003021A56E4F50C200F13BD
:101E0B009065777404F0906575E05401F0750A01E4
:101E1B00021A569080027410F0E4906577F090658A
:101E2B007504F0750AFA90668274FFF0021A5690E8
:101E3B006682E07003021EC19064757480F090643A
:101E4B00777401F0E4A3F0A304F0A37430F0A3744F
:101E5B007BF0E4F554747C2554F582E43464F5830B
:101E6B00747DF0747D2554F582E43464F583E4F0DD
:101E7B00E5542407906476F07C667D82906349E09C
:101E8B00FAA3E0FB7F021244A57E647F75E5542420
:101E9B0009FD124314906681E0601B124B09D203BB
:101EAB00E4F50A906575F090668604F0E490667927
:101EBB00F0A3F0021A56300F07E4906577F0800616
:101ECB009065777404F0750AFA021A5690800274C2
:101EDB0010F0750A05906575E06401FFF090657769
:101EEB007401F0EF7019906351E06013FCA3E0FDF7
:101EFB00A3E0FEA3E0FF906682122D4A021A5690D1
:101F0B00634DE0FCA3E0FDA3E0FEA3E0FF9066823F
:081F1B00122D4A021A5680FE45
:011F2300229B
:1008E100906376E0B444047F0180027F00906375D9
:1008F100E0B447047E0180027E00EE5F604A9063AF
:100901003EE0906377F090633FE0906378F090630E
:1009110040E0906379F0906341E090637AF09063F6
:1009210042E090637BF0906343E090637CF09063DE
:10093100767452F09062AE63A2019080A863A20126
:100941007F06122F2D02111A906331E0C3940850D3
:100951000302112390633EE0FF906377E06F600331
:1009610002112390633FE0FF906378E06F60030220
:100971001123906340E0FF906379E06F60030211FF
:1009810023906341E0FF90637AE06F6003021123DB
:10099100906342E0FF90637BE06F6003021123905C
:1009A1006343E0FF90637CE06F6003021123906377
:1009B10076E06444701A9080A8E0B4FF139062AEB0
:1009C10063A2019080A863A2017F06122F2D8010DF
:1009D1009062B2E09080ACF09062B3E09080ADF0B4
:1009E10090668BE060037401F090668C7464F09003
:1009F10063767452F0906375E0646D6003020B24BA
:100A01007BFF7A2479361228B27BFF7A24795090C1
:100A1100633EE0F55DA3E0F55EA3E0F55FA3E0F5DD
:100A210060A3E0F561A3E0F5621228B2755DFF7580
:100A31005E24755FAD7560FF7561247562B97BFFDA
:100A41007A2479861228B27BFF7A2479C21228B2DD
:100A51007BFF7A2579281228B27BFF7A2579559078
:100A61006344E0F55DA3E0F55EA3E0F55FA3E0F587
:100A7100601228B27BFF7A25797F90634DE0F55DA6
:100A8100A3E0F55EA3E0F55FA3E0F5601228B27B79
:100A9100FF7A2579AD906351E0F55DA3E0F55EA3A2
:100AA100E0F55FA3E0F5601228B27BFF7A2579DBE0
:100AB10090633AE0F55DA3E0F55EA3E0F55FA3E0A6
:100AC100F5601228B27BFF7A2579FE906336E0F556
:100AD1005DA3E0F55EA3E0F55FA3E0F5601228B247
:100AE1007BFF7A26791B1228B27BFF7A267944A2F2
:100AF1000FE433F55D1228B27BFF7A267974906694
:100B010081E0F55D1228B27BFF7A26799F90668B92
:100B1100E0F55D1228B21235007BFF7A2679D212F8
:100B210028B222906375E0644C70737E267FD8FBF7
:100B3100FDFC123A1890637DE0F555A3E0F556E40B
:100B4100F558E55590637FF0A3E556F07E277F13B6
:100B51007C637D7F7B02123A18E4F55785568285C6
:100B61005583E0FF747F2557F582E43463F583EF05
:100B7100F00556E556700205550557E557B410DCEA
:100B81007E277F167C637D7F7B10123A180558E51E
:100B910058C3941040AC7E277F19123C23229063E6
:100BA10075E0646C7060F5597E277F1BFBFDFC12BC
:100BB1003A18E4F558E490637FF0A3E559F07E27F5
:100BC1007F137C637D7F7B02123A18E4F557A859A5
:100BD100E6FF747F2557F582E43463F583EFF00572
:100BE100590557E557B410E67E277F167C637D7F54
:100BF1007B10123A180558E558C3940840B77E2770
:100C01007F19123C2322906375E0644B7061F557A4
:100C110074672557F582E43463F583E060327467C5
:100C21002557F582E43463F583E0F4602374672586
:100C310057F582E43463F583E0FF747D2557F5822F
:100C4100E43463F583E0B507100557E557B408C0F0
:100C51009061047432F002111A9063757421F030BE
:100C61000B0302111A7E277F56123C2302111A90A0
:100C71006375E0B4521A200B077E277F5E123C2376
:100C81009063757472F07E637F757D0812428D22C8
:100C9100906375E064497045200B077E277F6912D8
:100CA1003C2390637DE0F555A3E0F556E4F55785C7
:100CB1005682855583E0FF747F2557F582E43463BE
:100CC100F583EFF00556E556700205550557E557D2
:100CD100B480DC7E637F757D8A12428D22906375BC
:100CE100E064437046200B077E277F71123C2390FE
:100CF100637DE0F555A3E0F556E4F5578556828509
:100D01005583E493FF747F2557F582E43463F583BB
:100D1100EFF00556E556700205550557E557B480C5
:100D2100DB7E637F757D8A12428D22906375E0645C
:100D31005A7053200B077E277F7A123C2390637DE4
:100D4100E0F555A3E0F5567C637D7F7B80AF56AE21
:100D5100551249B7E4F557855682855583E493FFCB
:100D6100747F2557F582E43463F583EFF00556E58A
:100D710056700205550557E557B480DB7E637F75D4
:100D81007D8A12428D22906375E064446003020EF5
:100D91001890637DE0FF6444700302111AEFB431CF
:100DA1000CC20B7E277F86123C2302111A90637DB1
:100DB100E0B4300CD20B7E277F92123C2302111A31
:100DC10090637DE0B4320CD20C7E277F9F123C23CE
:100DD10002111A90637DE0B4330CC20C7E277FAD03
:100DE100123C2302111A90637DE0B4340CD20D7EC3
:100DF100277FBC123C2302111A90637DE0B4350CAD
:100E0100C20D7E277FC9123C2302111A90637DE037
:100E1100FF12002102111A906104E07013200B07E8
:100E21007E277FD7123C239063757421F002111A3B
:100E31009061047432F0906375E0FFB45104C2AF65
:100E410080FEEF64577045200B077E277FE5123C3B
:100E51002390637EE0906331F0E4F557906331E0D5
:100E6100FFE557C39F400302111A747F2557F5828E
:100E7100E43463F583E0FF90637DE0255724ADF50D
:100E810082E43461F583EFF0055780D0906375E01B
:100E910064536003020F3B200B077E277FF0123C57
:100EA1002390633EE0FF9061B6E06F703C90633F3A
:100EB100E0FF9061B7E06F7030906340E0FF9061B8
:100EC100B8E0B50724906341E0FF9061B9E0B50750
:100ED10018906342E0FF9061BAE0B5070C9063435C
:100EE100E0FF9061BBE06F60169063757421F03094
:100EF1000B0302111A7E277FFF123C2302111AE411
:100F0100F557E4F50DAF57FE74AD2557F582E4347E
:100F110061F583E0FD124A110557E557C394FE4080
:100F2100E1C2AFE4907FF0F0A3F0907FFD74AAF0EE
:100F3100A374FFF0A37455F080FE906375E0644FD5
:100F4100704C90637DE0F555A3E0F556E5564555A7
:100F5100700A200B077E287F08123C23200B077E96
:100F6100287F0F123C23E4F557747F2557F582E45F
:100F71003463F583E0855682855583F00556E55641
:100F8100700205550557E557B480DE02111A9063CA
:100F910075E0FFB4452190637DE0FDA3E0907FF013
:100FA100CDF0A3EDF0C2AF907FFD74AAF0A374FF62
:100FB100F0A37455F080FEEF646560030211239085
:100FC100637DE0FFA3E0907FF0CFF0A3EFF0E4F5C5
:100FD10055F556D3907FF1E09556907FF0E0955509
:100FE1004020E4F50D2556FFE5553401FE85568276
:100FF100855583E0FD124A110556E55670020555E7
:1010010080D17E287F1112439BEF4E602012000396
:10101100906344EFF0120003906345EFF012000378
:10102100906346EFF0120003906347EFF07E287F54
:101031001712439BEF4E602012000390634DEFF0B7
:1010410012000390634EEFF012000390634FEFF034
:10105100120003906350EFF07E287F1D12439BEF37
:101061004E6020120003906351EFF0120003906371
:1010710052EFF0120003906353EFF01200039063FC
:1010810054EFF07E287F2312439BEF4E6020120025
:101091000390633AEFF012000390633BEFF012000C
:1010A1000390633CEFF012000390633DEFF07E2864
:1010B1007F2912439BEF4E6020120003906336EFAD
:1010C100F0120003906337EFF0120003906338EFE2
:1010D100F0120003906339EFF0E4F557E4F50DE504
:1010E100572401FFE433FE74362557F582E4346357
:1010F100F583E0FD124A110557E557C3944340DCDF
:10110100C2AFE4907FF0F0A3F0907FFD74AAF0A34A
:1011110074FFF0A37455F080FE7E637F757D081225
:02112100428DFD
:0111230022A9
:10497F00AE07EEC39430400BEED394395005EE24BE
:10498F00D0FF22EEC39461400BEED394665005EE38
:10499F0024A9FF22EEC39441400BEED39446500559
:0849AF00EE24C9FF22AF06222D
:104AD7009062ADE004F070069062ACE004F0906282
:0A4AE700ACE0FEA3E0FF124A9D229E
:10000300124AD712497FEFC454F0FEC006124AD7F2
:0800130012497FD0E02FFF220B
:1047E100E4906BDEF0124AD7906BDFEFF0C39430A8
:1047F1004018E0FFD394395011906BDEE02405F5A9
:1048010082E43461F583EFF08011906BDEE02405E2
:10481100F582E43461F583E4F0800C906BDEE00412
:10482100F0E0D3940840BE755900755A00755B00DD
:0C483100E4F55C7B017A61790512303BF4
:01483D002258
:04439B008E5A8F5B4C
:10439F009062ACE4F0A374FFF0124AD7EF606EF4B2
:1043AF00606B855B82855A83E493B507EC755C017E
:1043BF00E55B255CF582E4355AF583E4936025903F
:1043CF0062ADE0255CFF9062ACE03400FE124A9DC6
:1043DF00E55B255CF582E4355AF583E493B5070474
:1043EF00055C80CCE55B255CF582E4355AF583E40A
:1043FF009370A6E55C24FFFFE434FFFE9062ADE00E
:10440F002FF09062ACE03EF07E007F0122E4FEFFD1
:01441F00227A
:103EC7007E287F2F12439BEF4E70037F01227E28AF
:103ED7007F3212439BEF4E600C124AD7EF24D02457
:103EE700FF920F8002D20F7E287F3812439BEF4E3E
:103EF700600C124AD7EF24D0906681F08005E490D9
:103F07006681F07E287F3E12439BEF4E600C124A7B
:103F1700D7EF24D090668BF08005E490668BF07E17
:103F2700287F4412439BEF4E600C124AD7EF24D0F0
:103F370024FF92018002C20190633E63A201906652
:103F47007B63A2017F06122F2D30013B7E287F4A1B
:103F570012439BEF4E603012000390667BEFF01226
:103F6700000390667CEFF012000390667DEFF0127D
:103F7700000390667EEFF012000390667FEFF01269
:0A3F87000003906680EFF07F002237
:1048F400906576E0C3947C503D906576E0FE04F0CC
:1049040074B42EF582E43462F583EFF0BF0A279085
:104914006576E0FF04F074B42FF582E43462F58325
:10492400E4F0906576E0FF1244209065767408F018
:074934009062B5E004F022DF
:10489A009080007480F090633663A201F583F582FC
:1048AA0063A2017F08122F2D90633E63A2019080BC
:1048BA008863A2017F0A122F2D9080927407F0A3B9
:1048CA0074D0F0A37406F0906348E0FF9080B1F0D2
:1048DA009080E1EFF09080957455F0A3F0908000FD
:0A48EA007401F090800974F0F022D0
:10471300908009E04410F09080A0E070609080A148
:104723007482F09080A874FFF0A3F0A3F0A3F07F4D
:10473300039080AEEFF0A374CBF09080007402F08E
:10474300906BD2122D5600000000906BD2E0908047
:1047530040F0906BD3E0908041F0906BD4E0908078
:1047630042F0906BD5E0908043F0A3E4F0A3F0A374
:0D477300F0A3F0908018F0A3F0A3F0A3F0E5
:014780002216
:10483E00908009E04440F09080D17482F07F039024
:10484E0080DEEFF0A374CCF09080027402F0906BD7
:10485E00D6122D5600000000906BD6E0908058F0D6
:10486E00906BD7E0908059F0906BD8E090805AF022
:10487E00906BD9E090805BF0A3E4F0A3F0A3F0A3DB
:0B488E00F0908030F0A3F0A3F0A3F046
:0148990022FC
:10462700908009E04420F09080B8E0706C9080B9E9
:104637007482F07F039080C6EFF07FCDA3EFF07F09
:10464700039080C4EFF0A374CDF09080C074FFF0A6
:10465700A3F0A3F0A3F09080017402F0906BDA123C
:104667002D5600000000906BDAE090804CF0906BC4
:10467700DBE090804DF0906BDCE090804EF0906B2B
:10468700DDE090804FF0A3E4F0A3F0A3F0A3F09057
:094697008024F0A3F0A3F0A3F0CD
:0146A00022F7
:1044A5008C558D56A907EAFDE975F018A424ACFFD3
:1044B500E5F034808F82F583EDF0EBFDE975F018BA
:1044C500A4FFAEF024ACFBEE34808B82F583A3ED24
:1044D500F08556828C83E0FDEF24A8FFEE3480FE44
:1044E5008F82F583EDF08556828C83A3E08F828ED3
:1044F50083A3F0855682855583A3A3E0FDE975F076
:1045050018A424A8FFE5F03480FE8F82F583A3A3C9
:10451500EDF08556828C83A3A3A3E08F828E83A3BF
:04452500A3A3F0223A
:06428D008D5AAB07AA06E2
:10429300908000E030E5079065787401F022906B20
:1042A300D2E0FCA3E0FDA3E0FEA3E0F55E8E5D8D0E
:1042B3005C8C5BAE02AF038E838F8263A201E55DEC
:1042C300540744C0F583855E8263A201AF5A122F5F
:1042D3009FE4FCFDFEE55E255AF55EEE355DF55D7A
:1042E300ED355CF55CEC355BF55B908040E55BF0B0
:1042F300A3E55CF0A3E55DF0A3E55EF090800074B8
:1043030020F0AF5EAE5DAD5CAC5B906BD2122D4A1C
:014313002287
:064314008D55AB07AA065F
:10431A00908002E030E5079065787403F022906B94
:10432A00D6E0FCA3E0FDA3E0FEA3E0F5598E588D8C
:10433A00578C56AE02AF038E838F8263A201E55873
:10434A00540744D0F58385598263A201AF55122FD1
:10435A009FE4FCFDFEE5592555F559EE3558F5580B
:10436A00ED3557F557EC3556F556908058E556F029
:10437A00A3E557F0A3E558F0A3E559F0908002743D
:10438A0020F0AF59AE58AD57AC56906BD6122D4AA5
:01439A002200
:023F91008F554A
:103F9300908001E030E5099065787402F07F00229B
:103FA300906BDAE0FCA3E0FDA3E0FEA3E0F5598EFD
:103FB300588D578C5690667B63A201E5585407448D
:103FC300C8F58385598263A2017F06122FB5E5598F
:103FD3002406F559E43558F558E43557F557E435D3
:103FE30056F55690657963A201E558540744C8F520
:103FF3008385598263A201AF55122FB5E4FCFDFE00
:10400300E5592555F559EE3558F558ED3557F5571A
:10401300EC3556F55690804CE556F0A3E557F0A3E2
:10402300E558F0A3E559F09080017420F0AF59AE44
:0D40330058AD57AC56906BDA122D4AAF55C0
:01404000225D
:103B1F009081E0E0F55505550555055505550555B9
:103B2F0005550555055505550555908010E0F55877
:103B3F00A3E0F559A3E0F55AA3E0F55B9081E1E02E
:103B4F00F5550555055505550555055505550555A6
:103B5F00055505550555908014E0F55CA3E0F55D1E
:103B6F00A3E0F55EA3E0F55FE55EB55A08E55FB546
:103B7F005B037F0022E4F555E55E540744E0F583CF
:103B8F00855F8263A20190637563A2017F08122F84
:103B9F00E590637763A2019062AE63A2017F061284
:103BAF002F2D906375E0F556A3E0F557E4F555908A
:103BBF006375E0702AA3E024F8F555E55E540744D9
:103BCF00E0F583855F8274082582F582E43583F5FD
:103BDF008363A20190637563A201AF55122FE5AE07
:103BEF0056E4FCFDE55F2557F55FE55E3EF55EEDBE
:103BFF00355DF55DEC355CF55C908014E55CF0A30C
:103C0F00E55DF0A3E55EF0A3E55FF0908000744002
:033C1F00F0AF55AE
:013C2200227F
:103379009081E6E0F5550555055505550555055561
:1033890005550555055505550555908028E0F5580D
:10339900A3E0F559A3E0F55AA3E0F55B9081E7E0D6
:1033A900F555055505550555055505550555055554
:1033B90005550555055590802CE0F55CA3E0F55DB4
:1033C900A3E0F55EA3E0F55FE4F555E55EB55A0ABD
:1033D900E55FB55B05C2080234E5E55E540744F0D4
:1033E900F583855F8263A20190637563A2017F08FB
:1033F900122FE5906375E0F556A3E0F557E55745BB
:103409005670099080027410F07F0022906682E065
:10341900FFF46030906377E06F60030234AC90662C
:1034290083E0FF906378E06F7079906684E0FF90A5
:103439006379E06F706D906685E0FF90637AE06F65
:103449006031805F906377E0906682F0906378E006
:10345900906683F0906379E0906684F090637AE0F7
:10346900906685F090637BE0FFA3E0906349CFF01D
:10347900A3EFF0906375E0702AA3E024F8F555E511
:103489005E540744F0F583855F8274082582F582CE
:10349900E43583F58363A20190637563A201AF5597
:1034A900122FE5AE56E4FCFDE55F2557F55FE55EB5
:1034B9003EF55EED355DF55DEC355CF55CAF5BAE1B
:1034C9005AAD59AC58AB5FAA5EA95DA85CD3122D61
:1034D9002640099080027410F07F002290802CE52C
:1034E9005CF0A3E55DF0A3E55EF0A3E55FF09080F5
:0634F900027440F0AF5523
:0134FF0022AA
:103675009081E3E0F5550555055505550555055565
:103685000555055505550555055590801CE0F5581A
:10369500A3E0F559A3E0F55AA3E0F55B9081E4E0DA
:1036A500F555055505550555055505550555055555
:1036B500055505550555908020E0F55CA3E0F55DC1
:1036C500A3E0F55EA3E0F55FE4F555E55EB55A0ABE
:1036D500E55FB55B05C2090237CBE55E540744E8F3
:1036E500F583855F8263A20190600463A2017F0E6A
:1036F500122FFB906004E0F556A3E0F55790600C9F
:10370500E0FFF4604A90667BE0FEEF6E7079A3E01F
:10371500FF90600DE06F706F90667DE0FF90600E2A
:10372500E06F706390667EE0FF90600FE06F70570A
:1037350090667FE0FF906010E06F704B906680E0D0
:10374500FF906011E06F703FE4906013F080089087
:10375500601374FFF0D2D9906004E0702AA3E024CE
:10376500F2F555E55E540744E8F583855F82740EEE
:103775002582F582E43583F58363A20190600463B5
:10378500A201AF55122FFBAE56E4FCFDE55F2557B0
:10379500F55FE55E3EF55EED355DF55DEC355CF5B9
:1037A5005CAF5BAE5AAD59AC58AB5FAA5EA95DA8DC
:1037B5005CD3122D265006E55745567009908001B9
:1037C5007410F07F0022908020E55CF0A3E55DF0A9
:1037D500A3E55EF0A3E55FF09080017440F0AF557E
:0137E50022C1
:043C23008E5A8F5BCB
:103C2700908000E030E5079065787401F022906B92
:103C3700D2E0FCA3E0FDA3E0FEA3E0F5618E608D7A
:103C47005F8C5EE561FFE5605407FEE42FF55DEEEE
:103C570034C0F55C855D82F5837423F0055DE55D11
:103C67007002055C535CC7F582855C83740AF005B6
:103C77005DE55D7002055C535CC790633E63A2011E
:103C8700855C83855D8263A2017F06122F9F740680
:103C9700255DF55DE4355CF55C855A83855B82635C
:103CA700A201855C83855D8263A201122F83E4FCF8
:103CB700FDFE906BD2E0F8A3E0F9A3E0FAA3E02FB2
:103CC700FFEE3AFEED39FDEC38FCEF2408FFE43E49
:103CD700FEE43DFDE43CFC906BD2122D4A906BD282
:103CE700E0908040F0906BD3E0908041F0906BD4EF
:103CF700E0908042F0906BD5E0908043F090800098
:033D07007420F035
:013D0A002296
:0A3A18008E5A8F5B8C5C8D5D8B5E17
:103A2200908000E030E5079065787401F022906B99
:103A3200D2E0FCA3E0FDA3E0FEA3E0F5648E638D7B
:103A4200628C61E564FFE5635407FEE42FF560EEE6
:103A520034C0F55F856082F5837423F00560E5600C
:103A62007002055F535FC7F582855F83740AF005B4
:103A720060E5607002055F535FC790633E63A20119
:103A8200855F8385608263A2017F06122F9F740681
:103A92002560F560E4355FF55F855A83855B826357
:103AA200A201855F8385608263A201122F838F65E5
:103AB200EF2560F560E4355FF55FE55E6017855CD4
:103AC20083855D8263A201855F8385608263A20133
:103AD200AF5E122F9FE5652408255EF55EFFE4FCCC
:103AE200FDFEE5642FF564EE3563F563ED3562F5B1
:103AF20062EC3561F561908040E561F0A3E562F02A
:103B0200A3E563F0A3E564F09080007420F0AF6455
:0C3B1200AE63AD62AC61906BD2122D4A24
:013B1E002284
:063DEC008E578F588D591F
:103DF200908000E030E5079065787401F022906BC6
:103E0200D2E0FCA3E0FDA3E0FEA3E0F55F8E5E8DB1
:103E12005D8C5CE55FFFE55E5407FEE42FF55BEE2B
:103E220034C0F55A855B82F5837423F0055BE55B4C
:103E32007002055A535AC7F582855A83EBF0055B27
:103E4200E55B7002055A535AC790633E63A201852F
:103E52005A83855B8263A2017F06122F9F74062517
:103E62005BF55BE4355AF55A85578385588263A220
:103E720001855A83855B8263A201AF59122F9F7419
:103E8200082559F559FFE4FCFDFEE55F2FF55FEECD
:103E9200355EF55EED355DF55DEC355CF55C90808B
:103EA20040E55CF0A3E55DF0A3E55EF0A3E55FF01D
:103EB2009080007420F0AF5FAE5EAD5DAC5C906B45
:043EC200D2122D4AA1
:013EC60022D9
:024420008F6E9D
:10442200908000E030E5079065787401F022906B8F
:10443200D2E0FCA3E0FDA3E0FEA3E0F5728E718D55
:10444200708C6FE572FFE5715407FEE42FFFEE34C6
:10445200C09062B463A201F5838F8263A201AF6E42
:10446200122F9FE4FCFDFEE572256EF572EE3571AA
:10447200F571ED3570F570EC356FF56F908040E5B4
:104482006FF0A3E570F0A3E571F0A3E572F0908000
:10449200007420F0AF72AE71AD70AC6F906BD2123F
:0244A2002D4AA1
:0144A40022F5
:063D0B008E598F5AAB0532
:103D1100908000E030E5079065787401F022906BA7
:103D2100D2E0FCA3E0FDA3E0FEA3E0F5608E5F8D91
:103D31005E8C5DE560FFE55F5407FEE42FF55CEE08
:103D410034C0F55B855C82F5837423F0055CE55C2A
:103D51007002055B535BC7F582855B83EBF0055C05
:103D6100E55C7002055B90633E63A201855B838520
:103D71005C8263A2017F06122F9F7406255CF55CAD
:103D8100E4355BF55B535BC7E559855C82855B83F5
:103D9100F0055CE55C7002055B535BC7F582855BF2
:103DA10083E55AF0055CE55C7002055B535BC7E592
:103DB10060240AF560E4355FF55FE4355EF55EE4A5
:103DC100355DF55D908040E55DF0A3E55EF0A3E52E
:103DD1005FF0A3E560F09080007420F0AF60AE5F0B
:0A3DE100AD5EAC5D906BD2122D4A6E
:013DEB0022B5
:104A9D00A2AF9210C2AF438E2075D2028F828E8349
:0C4AAD00E0FFE4F5D2538EDFA21092AFC0
:014AB90022DA
:104A1100E5D220E0FBA2AF9210C2AF43D2028F8257
:104A21008E83EDF075D25063D250A21092AFE5D2D1
:034A310020E0FB87
:014A3400225F
:1045A900E4FDED2401FFE433FE124A9D74362DF536
:1045B90082E43463F583EFF00DBD3FE6E4FDED24BD
:1045C9007FFFE433FE124A9D742D2DF582E4346198
:1045D900F583EFF0742D2DF582E43461F583E070F5
:1045E9001B742D2DF582E43461F5837420F0742E4B
:1045F9002DF582E43461F583E4F080040DBD80BEBD
:10460900E49061ACF0FDEDFF7E00124A9D74AD2D82
:0D461900F582E43461F583EFF00DBDFEE99C
:014626002271
:0249B7008B5A19
:1049B900A2AF9210C2AF85A25B53A2FE8E838F82F3
:1049C90005A28C838D827409123029E55A53A2FEFF
:1049D90043A22012302B53A2DF855BA2A21092AF13
:0149E900FFCE
:0149EA0022AA
:104ABA00A2AF9210C2AF8C838D82EF12302943A22B
:0C4ACA002012302B53A2DFA21092AFFF8D
:014AD60022BD
:024A35008F559B
:104A3700A2AF9210C2AFE4F5838D827406123029BB
:104A4700E55543A22012302B53A2DFA21092AF7F6D
:014A5700015D
:014A5800223B
:024A59008F5577
:104A5B00A2AF9210C2AFE4F5838D82740A12302993
:104A6B00E55543A22012302B53A2DFA21092AF7F49
:014A7B000139
:014A7C002217
:102E5200A907E7FFA805EF93C3966008403B74FCFF
:102E62002FFF80F00F08EF93C3966008402B74FB8E
:102E72002FFF80E00F08EF93C3966008401B74FA9F
:102E82002FFF80D00F08EF93D3966008400B74F9A0
:102E92002FFF80C01F1F1F1F1FEF54FEF80303F7F1
:102EA200E893FC08E893FD08E893FE08E893FF2204
:102EB20009E993C39D6008402974FB29F980F1094F
:102EC200E993C39E6008401A74FA29F980E209E97D
:102ED20093D39F6008400B74F929F980D31919190B
:102EE2001919E9C313C313FF22740093F8ECC398B2
:102EF2004024701F740193F8EDC398401970147444
:0E2F02000293F8EEC398400E7009740393F822
:102F1000EFC39840037F00227F0122EDF8E6F0081E
:102F2000A3DFFA22EDF8E0F608A3DFFA22E0A363BC
:102F3000A201F0A363A201DFF475A2002263A20143
:102F4000F0A363A20122E0A363A201F0A363A201A4
:102F5000E0A363A201F0A363A201E463A201F0A3D2
:102F600063A201DFE175A20022E0A363A2016DFE6E
:102F7000936CFDEE058393FC158363A201DFEA7574
:102F8000A200227F00E493A363A201F00F600CA3D0
:102F9000E583C2E3F58363A20180EA75A20022E023
:102FA000A363A201F0A3E583C2E3F58363A201DF7B
:102FB000EE75A20022E0A363A201F0A3E583C2E4C0
:102FC000D2E3F58363A201DFEC75A20022E0A363E4
:102FD000A201F0A3E58344F8C2E5F58363A201DF13
:102FE000EC75A20022E583C2E3F583E0A363A201AE
:102FF000F0A363A201DFEE75A20022E583C2E4D252
:0A300000E3F583E0A363A201F0A34F
:10300A0063A201DFEC75A20022E58344F8F583E0B0
:10301A00A363A201F0A363A201DFEE75A20022F965
:10302A0022C002C004C00612FFF0D006D004D002AB
:01303A002273
:101F24003E2A2C312CCFE0F0E0ECE5F2F0FB20F877
:101F3400E8EDFB2043414E0A003E4C2C6B30312C23
:101F440025732C43EAEEF0EEF1F2FC20EDE020F8EC
:101F5400E8EDE52043414E2C30202D20353030EA89
:101F6400E1283530EC292C31202D203530EAE128C8
:101F7400353030EC290A0030202D20353030EAE1AC
:101F8400283530EC290031202D203530EAE1283580
:101F94003030EC29003E2A2C312CCFE0F0E0ECE587
:101FA400F2F0FB20EFF0EEF2EEEAEEEBE020D1DD12
:101FB400D22D34D2CC28CCE5F0EAF3F0E8E9323380
:101FC40030290A003E422C4930322C2562752CD22D
:101FD400E8EF20EFF0EEF2EEEAEEEBE020CCE5F0F5
:101FE400EAF3F0E8E90A003E532C4930332C257318
:101FF4002CCFE0F0EEEBFC20E4EEF1F2F3EFE00A9C
:10200400003E4C2C4930312C256C752CD1EAEEF075
:10201400EEF1F2FC20EEE1ECE5EDE02C3132303073
:102024002C323430302C343830302C393630302C9B
:1020340031393230300A003E422C4930352C256289
:10204400752CCAEEEDF2F0EEEBFC20EFEE20EDE5A0
:10205400F7E5F2EDEEF1F2E80A003E532C49313295
:102064002C2562752CC0E4F0E5F120E1EBEEEAE00A
:1020740020D2C8D220EDE020F8E8EDE50A003E5376
:102084002C4931332C25752CCFE0F3E7E020ECE527
:10209400E6E4F320F6E8EAEBE0ECE828F1E5EA29E7
:1020A4000A003E532C6D2562752C25732CCFF0E865
:1020B400E1EEF0202562752028C0E4F0E5F120E887
:1020C40020EFE0F0E0ECE5F2F0FB290A003C21000F
:1020D4003C6B30313D003C4930333D003C493031AC
:1020E4003D003C4931323D003C4931333D003C49DF
:1020F40030323D003C4930353D002043616E45722D
:1021040047495400200A002043616E4572724348D7
:1021140021000A000AC7E0EFF0EEF13A00CFF0E840
:10212400E5EC3A00CEF8E8E1EAE020CAD1210A0061
:10213400CED8C8C1CAC020C0E4F0E5F1E02100CE89
:10214400D8C8C1CAC020EEF2EAF0FBF2E8FF20EAE8
:10215400E0EDE0EBE02100204F4B212000CED8C879
:10216400C1CAC020E7E0EFF0EEF1E0000A3D00282C
:10217400253033642920256C642020202020202051
:1021840020202020200000C1814001C0804101C0E6
:10219400804100C1814001C0804100C1814000C133
:1021A400814001C0804101C0804100C1814000C123
:1021B400814001C0804100C1814001C0804101C013
:1021C400804100C1814001C0804100C1814000C103
:1021D400814001C0804100C1814001C0804101C0F3
:1021E400804100C1814000C1814001C0804101C0E3
:1021F400804100C1814001C0804100C1814000C1D3
:10220400814001C0804101C0804100C1814000C1C2
:10221400814001C0804100C1814001C0804101C0B2
:10222400804100C1814000C1814001C0804101C0A2
:10223400804100C1814001C0804100C1814000C192
:10224400814001C0804100C1814001C0804101C082
:10225400804100C1814001C0804100C1814000C172
:10226400814001C0804101C0804100C1814000C162
:10227400814001C0804100C1814001C0804101C052
:10228400804100C1814000C0C101C30302C2C6062F
:1022940007C705C5C404CC0C0DCD0FCFCE0E0ACA9A
:1022A400CB0BC90908C8D81819D91BDBDA1A1EDEEA
:1022B400DF1FDD1D1CDC14D4D515D71716D6D2129A
:1022C40013D311D1D010F03031F133F3F23236F6AA
:1022D400F737F53534F43CFCFD3DFF3F3EFEFA3A5A
:1022E4003BFB39F9F83828E8E929EB2B2AEAEE2EEA
:1022F4002FEF2DEDEC2CE42425E527E7E62622E25A
:10230400E323E12120E0A06061A163A3A26266A6A9
:10231400A767A56564A46CACAD6DAF6F6EAEAA6A19
:102324006BAB69A9A86878B8B979BB7B7ABABE7E69
:102334007FBF7DBDBC7CB47475B577B7B67672B219
:10234400B373B17170B050909151935352929656A9
:102354005797559594549C5C5D9D5F9F9E5E5A9AD9
:102364009B5B99595898884849894B8B8A4A4E8E69
:102374008F4F8D4D4C8C44848545874746868242D9
:102384004383418180403C6D303D000000003C6D42
:10239400313D000000003C6D323D000000003C6D0A
:1023A400333D000000003C6D343D000000003C6DF6
:1023B400353D000000003C6D363D000000003C6DE2
:1023C400373D000000003C6D383D000000003C6DCE
:1023D400393D000000003C6D31303D0000003C6D93
:1023E40031313D0000003C6D31323D0000003C6D58
:1023F40031333D0000003C6D31343D0000003C6D44
:0624040031353D0000002F
:0100210022BC
:030023000246A1F1
:0B46A100C0E0C083C082C0D075D018FC
:1046AC00309827E5E92464F5EB30D707E5F904F5F4
:1046BC00FB800385F9FBD29174AA253DF582E43485
:1046CC006AF583E599F0053DC298309931E542C30E
:1046DC00953C501BAF42054274AA2FF582E4346B13
:1046EC00F583E0FF521FA2D0B3929B8F99800DE50A
:0E46FC0042C3953C40060542D296C290C29938
:09470A00D0D0D082D083D0E0327F
:103500007BFF7A1F79241228B290688DE0701475C1
:103510005DFF755E1F755F7B7BFF7A1F793D12280B
:10352000B28012755DFF755E1F755F8A7BFF7A1F23
:10353000793D1228B27BFF7A1F79991228B27BFF5E
:103540007A1F79C8A21DE433F55D1228B2755D01BA
:10355000755E6A755F5F7BFF7A1F79EB1228B29008
:103560006BCCE0FEA3E0FFC3E49FFFE49EFEAB074D
:10357000FA3395E0F9F87F007E8C7D0A7C00122CEE
:10358000868F608E5F8D5E8C5D7BFF7A2079051261
:1035900028B27BFF7A20793BA219E433F55D12282B
:1035A000B27BFF7A20795E90688EE0F55D1228B2DA
:1035B000E47B64FAF9F8AF37AE36AD35AC34122C93
:1035C000868F608E5F8D5E8C5D7BFF7A20798212A4
:1035D00028B2E4906BDEF0906BDEE0FFC364809471
:1035E000904003023674906A0E7420F0E4A3F0EF6A
:1035F0003395E0FEEF7803C333CE33CED8F9248A77
:10360000F58274233EAF82FE12439BEF4E6041E48D
:10361000906BE0F0124AD7906BDFEFF0643C601BD8
:10362000E0FFA3E0FE04F0EEFD3395E0FC740E2D08
:10363000F582746A3CF583EFF080D9906BE0E0FF8F
:103640003395E0FE740E2FF582746A3EF583E4F044
:10365000906BDEE0F55D755E01755F6A75600E0466
:10366000F5617BFF7A2079A61228B2906BDEE00428
:04367000F00235D758
:013674002233
:06493B00AC05AB07AA0663
:10494100906A0D74FFF0906A5EF0AF041CEF602D69
:104951000BEBAE0270010A14F5828E83E0FF906AC0
:104961000DE06FFF90218A93FE906A5EE06E906A7F
:0D4971000DF0EF90228A93906A5EF080CDE9
:01497E002216
:04452900A907AE032D
:10452D00E4906BDEF0906BDEE0FFC39440501B8592
:10453D004982854883A3E5822FF582E43583F5838F
:10454D00E4F0906BDEE004F080DB854982854883E2
:10455D007406F0A3E9F0854982854883A3A3740806
:10456D00F0EED39401400E854982854883A3A3A321
:10457D007416F0800C854982854883A3A3A3741417
:10458D00F0E5492404F582E43548F583EDF0E5497D
:0B459D00241CF582E43548F583EEF0A5
:0145A80022F0
:100026007E207FD112439BEF4E70037F0122E49026
:10003600688DF07E207FD412439BEF4E601B124AE0
:10004600D78F55E555B4310690688D740AF0E5559D
:10005600B4320690688D7464F07E207FDA12439B7A
:10006600EF4E6035124AD7906A5FEFF0124AD7908A
:100076006A60EFF0124AD7906A61EFF0124AD790A1
:100086006A62EFF0124AD7906A63EFF0124AD7908D
:100096006A64EFF0E4A3F08013906A5F7431F0A312
:1000A600F0A3F0A3F0A3F0A3F0E4A3F07E207FE09A
:1000B60012439BEF4E60231247E1A804A905AA0646
:1000C600AB077F007E8C7D0A7C00122C86122D18D1
:1000D600906BCCEEF0A3EFF0800A906BCC74FFF03F
:1000E600A374B8F07E207FE612439BEF4E600A129F
:1000F60047E190688EEFF08005E490688EF07E20F0
:100106007FEC12439BEF4E60161247E1E47B64FAE4
:10011600F9F8122BFB8F378E368D358C348009E437
:10012600F537F536F535F534E4FFFEFDFCAB37AAB9
:1001360036A935A834C3122D26700975370AF53647
:10014600F535F5347E207FF212439BEF4E600D129B
:1001560047E1EC4D4E4F24FF921D8002C21D7E20CA
:100166007FF812439BEF4E600C124AD7EF24D0243F
:10017600FF92198002C219E4F548F549301D5F85E2
:100186004982854883A374FEF0854982854883A306
:10019600A37403F0854982854883A3A3A37408F05A
:1001A600E5492401FFE43548FE7D0312493B906A88
:1001B6000DE0FFE5492404F582E43548F583EFF0C8
:1001C600906A5EE0FFE5492405F582E43548F5834B
:1001D600EFF08549828548837405F00202788549E7
:1001E60082854883A374FEF0854982854883A3A34C
:1001F6007403F0854982854883A3A3A37408F0E5B8
:10020600492404F582E43548F5837455F0E549241C
:1002160005F582E43548F58374AAF0E5492406F528
:1002260082E43548F5837433F0E5492407F582E422
:100236003548F58374CCF0E5492401FFE43548FEE2
:100246007D0712493B906A0DE0FFE5492408F582D7
:10025600E43548F583EFF0906A5EE0FFE54924094E
:10026600F582E43548F583EFF08549828548837445
:1002760009F074202549F549E43548F54885498251
:10028600F583E4F0906A0C04F0E4F555AF55EF33CE
:1002960095E0FEEF7803C333CE33CED8F9248AF542
:1002A6008274233EAF82FE12439BEF4E7003020818
:1002B6002C1247E1906AA9EFF0700302083A906A9F
:1002C600A9E0B4FF02E4F0201D0302039E906AA990
:1002D600E0854982854883A3F0854982854883A3C2
:1002E600A37401F0854982854883A3A3A3F0906A8D
:1002F6005FE0FFE5492404F582E43548F583EFF035
:10030600906A60E0FFE5492405F582E43548F58307
:10031600EFF0906A61E0FFE5492406F582E435488E
:10032600F583EFF0906A62E0FFE5492407F582E481
:100336003548F583EFF0906A63E0FFE5492408F558
:1003460082E43548F583EFF0906A64E0FFE54924DE
:1003560009F582E43548F583EFF0E5492401FFE429
:100366003548FE7D0912493B906A0DE0FFE54924B8
:100376000AF582E43548F583EFF0906A5EE0FFE522
:1003860049240BF582E43548F583EFF085498285EB
:100396004883740BF0020458906AA9E08549828567
:1003A6004883A3F0854982854883A3A37401F0900E
:1003B6006A5FE0854982854883A3A3A3F0906A60BB
:1003C600E0FFE5492404F582E43548F583EFF09033
:1003D6006A61E0FFE5492405F582E43548F583EFD7
:1003E600F0906A62E0FFE5492406F582E43548F5B7
:1003F60083EFF0906A63E0FFE5492407F582E43570
:1004060048F583EFF0906A64E0FFE5492408F58239
:10041600E43548F583EFF0E5492401FFE43548FE6D
:100426007D0812493B906A0DE0FFE5492409F582F3
:10043600E43548F583EFF0906A5EE0FFE549240A6B
:10044600F582E43548F583EFF08549828548837463
:100456000AF0E549241CF582E43548F583E4F07496
:10046600202549F549E43548F548906A0CE004F042
:10047600854982854883E4F0124AD7EF122D870515
:100486006D00056D2104CE23081A2A07CF2F04ED2F
:100496003B056D3C07CF3E06924306A14506324614
:1004A60006714906624C05F65006055107E65206E6
:1004B6002353064155074B6107776207A36306E19D
:1004C600650721730000047E124AD775F008EFA471
:1004D6002402F582E5F03422AF82FE12439BEF4EF2
:1004E60060961247E18091E5492401FFE43548FE14
:1004F6007D0412493B906A0DE0FFE5492405F5822B
:10050600E43548F583EFF0906A5EE0FFE54924069E
:10051600F582E43548F583EFF0E5492401FFE4353B
:1005260048FE7D0612493B906A0DE0FFE549240727
:10053600F582E43548F583EFF0906A5EE0FFE54921
:100546002408F582E43548F583EFF074202549F553
:1005560049E43548F548906A0CE004F085498285FF
:100566004883E4F002047E854982854883E060750D
:10057600E5492401FFE43548FE7D0412493B906AB3
:100586000DE0FFE5492405F582E43548F583EFF0F3
:10059600906A5EE0FFE5492406F582E43548F58376
:1005A600EFF0E5492401FFE43548FE7D0612493B9C
:1005B600906A0DE0FFE5492407F582E43548F583A6
:1005C600EFF0906A5EE0FFE5492408F582E43548DD
:1005D600F583EFF074202549F549E43548F5489050
:1005E6006A0CE004F0854982854883E4F002082C11
:1005F600906AA9E0FF7B0FE4FD12452902047E9074
:100606006AA9E0FF7B0F7D04124529E549241EF502
:1006160082E43548F583E04410F002047E906AA92E
:10062600E0FF7B0F7D0812452902047E906AA9E04F
:10063600FF7B017D4012452902047E301D0F906A22
:10064600A9E0FF7B077D1112452902047E906AA965
:10065600E0FF7B0E7D1012452902047E906AA9E018
:10066600FF7B0E7D1412452902047E301D0F906A11
:10067600A9E0FF7B077D2112452902047E906AA925
:10068600E0FF7B0E7D2012452902047E906AA9E0D8
:10069600FF7B0F7D3012452902047E906AA9E0FF98
:1006A6007B017D0F124529854982854883A3A37462
:1006B60005F0854982854883A3A3A3E4F0E5492490
:1006C60004F582E43548F583E4F0E549241CF58217
:1006D600E43548F583740FF002047E906AA9E0FFC2
:1006E6007B017D0F124529854982854883A3A37422
:1006F60005F0854982854883A3A3A3E4F0E5492450
:1007060004F582E43548F583E4F0E549241CF582D6
:10071600E43548F5837405F002047E8549828548F0
:1007260083A3A3A37411F0E5492404F582E43548B4
:10073600F583E0F0E549241CF582E43548F5837439
:1007460001F002047E854982854883A3A3A3741120
:10075600F0E5492404F582E43548F583E04401F0E8
:10076600E549241CF582E43548F5837401F002045A
:100776007E854982854883A3A3A37411F0E54924A5
:1007860004F582E43548F583E04402F0E549241C8B
:10079600F582E43548F5837401F002047E854982CA
:1007A600854883A3A3A37411F0E5492404F582E4E4
:1007B6003548F583E04403F0E549241CF582E43529
:1007C60048F5837401F002047E124AD7EF24D0FF65
:1007D600E549241DF582E43548F583EFF002047EF1
:1007E600E549241EF582E43548F583E0FF30E4123E
:1007F600E549241EF582E43548F583EF4440F002CE
:10080600047EE549241EF582E43548F583E044017B
:10081600F002047EE549241EF582E43548F583E0BE
:100826004402F002047E0555C3E555648094905059
:1008360003020292E4F548F549FFF555854982859C
:100846004883E070030208DAA3A3E06408703EE57B
:1008560049241FF582E43548F583E555F0E549243A
:100866001CF582E43548F583E0FEB401020555EE39
:10087600B40F0674042555F555EEB40E067403251B
:1008860055F555EEB4070674032555F55585498289
:10089600854883A3A3E06405702CE549241FF582EF
:1008A600E43548F583EFF0E549241CF582E4354844
:1008B600F583E0FEB401010FEEB40F0474042FFFBC
:1008C600EEB405020F0F74202549F549E43548F5C5
:0A08D60048020842E4F548F549FF26
:0108E00022F5
:1049EB00C2A9438902758C48758A4875D90475DB51
:1049FB004875DC4875DD4875DE48E4F5E9F5F9C224
:064A0B00D9D28CD2DE229C
:1040DF0043AB01C2E8C2EAE4FFEFC454F0F5B1C349
:1040EF00EF64809488500575B3D08003E4F5B3EF87
:1040FF007026F5B275BC01F5BDF5BEF5BF75C4FFF1
:10410F00F5C5F5C6F5C7F5A3F5A3F5A3F5A3F5A377
:10411F00F5A3F5A3F5A38027E4F5B275BCC8F5BDEB
:10412F00F5BE75BF7875C4FFF5C5F5C675C778F5CB
:10413F00A3F5A3F5A3F5A3F5A3F5A3F5A3F5A30F96
:10414F00BF0E9690688DE0FF25E0F5B475B50C7540
:10415F00B66C75A11275AB0275C13E75C3FF75C202
:01416F00034C
:01417000222C
:1047810075B180E4F5B3F5B28527BCE5285403FF84
:1047910033333354F8FFE52854E04FFFE529C413C0
:1047A10054074FF5BDE52933333354F8FFE52AC4E7
:1047B1001354074FF5BEE52A33333354F8F5BF855B
:1047C1002CA3852DA3852EA3852FA38530A3853109
:1047D100A38532A38533A3E52B540F2450F5B322CF
:10390B00E59B541F6020200B1A7E207FFE123C2368
:10391B00E59B541FFF7E007D03123D0B7E217F082C
:10392B00123C23E4F59BE5BA30E008E4F5B375B13E
:10393B0080F5B2E5CFF47003023A15755801E4F542
:10394B0057E5CFF455587003023A03E557C454F0CA
:10395B00F5B1E5B2547F6420706FE5B3540FF52BCE
:10396B0085BC27E5BD541FFF131313541FFFE5BD83
:10397B0054E044184FF528E5BDC43354E0FFE5BED1
:10398B00131313541F4FF529E5BEC43354E0FFE561
:10399B00BF131313541F4FF52A85A32C85A32D8515
:1039AB00A32E85A32F85A33085A33185A33285A3B1
:1039BB0033E4F5B2E527547EB5270575B350800384
:1039CB0075B3D0E52B2405FF22E5B2549F6023206D
:1039DB000B207E217F0B123C23AFB27E007D0312A6
:1039EB003D0BAFB37E007D03123D0B7E217F161284
:1039FB003C23E4F5B275B3D0E55825E0F5580557EF
:0C3A0B00E557C39408500302394C7F00BB
:013A1700228C
:10404100C21AE4F53DF50BD296F53CF542F525FF94
:1040510074692FF582E4346AF583E4F074912FF5E5
:1040610082E43468F583E4F00FBF40E4E49069D85A
:10407100F0A3F0F543F5531200261240DFC2ADE480
:10408100F5C9D2CDD2CCC2C9C2CAF5CDF5CC906B9F
:10409100CCE0F5CBA3E0F5CA85CBCD85CACCE4F560
:1040A100985387BF301906D29FD29E8002D29E4379
:1040B1008740C29FC2ACC298C29975B81075B7103B
:1040C100D2CAD29CD2AC1249EBC2D9E5E92464F53B
:0D40D100EB30D706E5F904F5FB2285F9FB7D
:0140DE0022BF
:0100220022BB
:014B0800228A
:014B09002289
:104A7D00906379E0B40118906381E0F54A9063800A
:104A8D00E0F54B90637FE0F54C90637EE0F54D22B1
:1031DF00AF37AE36AD35AC34EC4D4E4F6007E546EC
:1031EF0070037F0122854982854883E07024F5486A
:1031FF00F549AF37AE36AD35AC34EC4D4E4F6006BA
:10320F00E4F5467F0122854982854883E070037F7C
:10321F000122854982854883A3A3E0640170537519
:10322F00390185483A85493BE549241CF582E43547
:10323F0048F583E0601674202549F549E43548F5D3
:10324F0048854982F583E0709C7F0122E54924017E
:10325F00FFE43548F5838F8263A201906BAA63A2C6
:10326F00017F0C122F2D854982854883E0F53C02A2
:10327F00335B854982854883A3A3E0FF6403600322
:10328F00EF7032052553250FE49069D8F0A3F0E5D0
:10329F00492401FFE43548F5838F8263A201906BC7
:1032AF00AA63A2017F0C122F2D854982854883E0E6
:1032BF00F53C02335BAB39AA3AA93B90001C122BA9
:1032CF00AC700E74202549F549E43548F5480231B4
:1032DF00F4E549241EF582E43548F583E030E11228
:1032EF00E525600E74202549F549E43548F5480277
:1032FF0031F4854982854883A3E0906BAAF0854914
:10330F0082854883A3A3E0906BABF0854982854803
:10331F0083A3A3A3E0906BACF0E5492404F582E40A
:10332F003548F583E0906BADF0E5492405F582E46F
:10333F003548F583E0906BAEF0E5492406F582E45D
:10334F003548F583E0906BAFF0753C06E4F542D25B
:10335F0090C291C296D299200B0D7E217F187C6B63
:09336F007DAAAB3C123A187F0064
:013378002232
:1037E600E553C394404003E4F553E538C3944040A1
:1037F60003E4F53874912538F582E43468F583E0FE
:10380600FF30E17B74912538F582E43468F583EF67
:1038160054FDF0E4906475F0A3740DF090667AE0C0
:10382600906477F0A37419F0A37444F0A37439F08C
:10383600E538C4135407FF90688EE02F90647BF040
:10384600E538541F04A3F0A37408F0E53825E025F5
:10385600E024D8F582E43468F58363A20190647E9F
:1038660063A2017F04122F2D906482E54DF0A3E53B
:103876004CF0A3E54BF0A3E54AF005387F0122742E
:10388600692553F582E4346AF583E0FF30E16F740D
:10389600692553F582E4346AF583EF54FDF0E4902C
:1038A6006475F0A3740DF090667AE0906477F0A3E7
:1038B6007419F0A37448F0A37479F0E55313131345
:1038C600541FFF90688EE02F90647BF0E5535407F9
:1038D60025E025E02480A3F0A37408F0F5F0E55375
:1038E600A4248DF582E5F03466F58363A201906425
:1038F6007E63A2017F08122F2D05537F01220553F7
:0539060005387F0022DE
:014B0A002288
:1011240074692543F582E4346AF583E020E002051E
:1011340043E543C394404003E4F54374912524F507
:1011440082E43468F583E020E0020524E524C394B6
:10115400404003E4F52412390BEF7003021247E513
:1011640027B4010C852F4A852E4B852D4C852C4D9B
:10117400E52A640F600302124790688EE0FF652938
:10118400600302124774912524F582E43468F583E0
:10119400E0FE30E05174912524F582E43468F5834F
:1011A400EE54FEF0752744752839E524C41354071A
:1011B400FEEF2EF529E524541F04F52A752B08E5C6
:1011C4002425E025E024D8F582E43468F5837D2CD9
:1011D4007F04122F24854D30854C31854B32854A4E
:1011E40033124781805D74692543F582E4346AF5DE
:1011F40083E0FF30E04D74692543F582E4346AF5F9
:1012040083EF54FEF0752748752879E543131313CB
:10121400541FFF90688EE02FF529E543540725E01D
:1012240025E02480F52A752B0875F008E543A424ED
:101234008DF582E5F03466F5837D2C7F08122F242A
:10124400124781200203021357C202054EE54EC322
:1012540094644066E4F54EAF4DAE4CAD4BAC4AFAE7
:10126400F9F8EF2401F54DEA3EF54CE93DF54BE87C
:101274003CF54AE47B3CAF4DAE4CAD4BAC4A122C32
:1012840086AC00AD01AE02AF03E4FBFAF9F8C31279
:101294002D267026F55574912555F582E43468F5AC
:1012A40083E030E20E74912555F582E43468F583C9
:1012B4007403F00555E555B440DCE546704E90687E
:1012C400D3E0FCA3E0FDA3E0FEA3E0FFE4FAF9F819
:1012D400EF2401FFEA3EFEE93DFDE83CFC9068D3C3
:1012E400122D4AAF37AE36AD35AC349068D3E0F842
:1012F400A3E0F9A3E0FAA3E0FBC3122D26400D7589
:1013040046019068D3122D5600000000906890E0CA
:1013140004F0700690688FE004F0D3906890E09435
:10132400B890688FE0940B402AE4F0A3F0F555746C
:10133400692555F582E4346AF583E030E20E746978
:101344002555F582E4346AF5837403F00555E555B3
:10135400B440DC20D9030218BAC2D9E53DD39400C5
:101364005003021853C291853D47E4F53DF50B7EC9
:101374006A7FAAAD4712493B200B0D7E217F217C59
:101384006A7DAAAB47123A18906A5EE0FF906A0D34
:10139400E04F6010300B030218537E217F28123C6B
:1013A40023021853854982854883A3E0FF906AAAE3
:1013B400E06F6010300B030218537E217F34123C1F
:1013C40023021853854982854883A3A3E0640170EE
:1013D4003D906AABE0601A200B077E217F43123CEC
:1013E40023E549241CF582E43548F583E4F002182A
:1013F40053D21B200B077E217F5B123C23E549243B
:101404001CF582E43548F5837401F0021853D21BAD
:10141400E547C39406501DAB39AA3AA93B90001C7A
:10142400E4122BD9300B030218537E217F61123C46
:1014340023021853854982854883A3A3E0B4081C7A
:10144400E549241FF582E43548F583E075F002A4EC
:10145400FF9069D8E5F0F0A3EFF0801AE549241F66
:10146400F582E43548F583E075F004A4FF9069D86B
:10147400E5F0F0A3EFF0E4F555E549241CF582E42A
:101484003548F583E0FD7C0074017E00A855088092
:1014940005C333CE33CED8F9FFEE5CFEEF5D4E705C
:1014A40003021847854982854883A3A3E064086042
:1014B40003021694301D41E55575F003A424ABF5E1
:1014C40082E4346AF583E0F556E4F53EE556543F8C
:1014D400F53FE55575F003A424ADF582E4346AF5CF
:1014E40083E0F540E55575F003A424ACF582E434BB
:1014F4006AF583E0F541803FE55575F003A424AB1C
:10150400F582E4346AF583E0F556E4F53EE5565495
:101514003FF53FE55575F003A424ACF582E4346A45
:10152400F583E0F540E55575F003A424ADF582E4B8
:10153400346AF583E0F541AF41AE40AD3FAC3EE5E2
:1015440049241DF582E43548F583E0F9F8122D3776
:101554008F418E408D3F8C3EE55630E71AE5492495
:101564001EF582E43548F583E030E00BC3E4954191
:10157400F541E49540F540E55630E61AE549241E68
:10158400F582E43548F583E030E60BC3E49541F594
:1015940041E49540F540300C417E217F70123C239C
:1015A400755DFF755E21755F739069D8E0C313F5AF
:1015B40060A3E013F561AF41AE40AD3FAC3E8F6533
:1015C4008E648D638C627B017A6979DA1228AC7E31
:1015D400697FDA7B057D0F123DEC9069D8E0FEA3AC
:1015E400E0248DF58274663EF583E06541602990C0
:1015F40069D8E0A3E0FF248DF58274663EF583E5A7
:1016040041F0EF7803CEC313CE13D8F92469F582E1
:10161400746A3EF5837407F09069D9E004F07006AB
:101624009069D8E004F09069D8E0FCA3E0FD248D33
:10163400F58274663CF583E06540602A9069D8E0E1
:10164400FEA3E0FF248DF58274663EF583E540F049
:10165400EF7803CEC313CE13D8F92469F582746AE4
:101664003EF5837407F0EDAE047803CEC313CE13B6
:10167400D8F92469F582746A3EF583E04404F09055
:1016840069D9E004F070069069D8E004F0021847C4
:10169400201D03021772E55525E025E024ADF582EF
:1016A400E4346AF583E0FF9069D9E024D8F582E454
:1016B4003468F583EFF09069D9E004F0700690691E
:1016C400D8E004F0E55525E025E024AEF582E434C5
:1016D4006AF583E0FF9069D9E024D8F582E43468A0
:1016E400F583EFF09069D9E004F070069069D8E0D2
:1016F40004F0E55525E025E024ABF582E4346AF5F1
:1017040083E0FF9069D9E024D8F582E43468F58356
:10171400EFF09069D8E0FEA3E07802CEC313CE13B5
:10172400D8F92491F58274683EF583E04404F0907E
:1017340069D9E004F070069069D8E004F0E5552515
:10174400E025E024ACF582E4346AF583E0FF906997
:10175400D9E024D8F582E43468F583EFF09069D9B0
:10176400E004F070069069D8E004F0021847E555EB
:1017740025E025E024AEF582E4346AF583E0FF90A9
:1017840069D9E024D8F582E43468F583EFF09069F0
:10179400D9E004F070069069D8E004F0E55525E03E
:1017A40025E024ADF582E4346AF583E0FF9069D93D
:1017B400E024D8F582E43468F583EFF09069D9E049
:1017C40004F070069069D8E004F0E55525E025E0C2
:1017D40024ACF582E4346AF583E0FF9069D9E0240F
:1017E400D8F582E43468F583EFF09069D8E0FEA37D
:1017F400E07802CEC313CE13D8F92491F58274682D
:101804003EF583E04404F09069D9E004F07006905A
:1018140069D8E004F0E55525E025E024ABF582E441
:10182400346AF583E0FF9069D9E024D8F582E43482
:1018340068F583EFF09069D9E004F070069069D8F8
:10184400E004F00555E555C39404500302147D20CB
:101854001B0DAB39AA3AA93B90001CE4122BD9E525
:101864003C600FE546600B74202549F549E4354892
:10187400F548E5E924E8F5EB30D708E5F92404F563
:10188400FB8006E5F92403F5FB1231DFEF702785B1
:101894004982854883A3A3E0B40319E5E924F4F558
:1018A400EB30D708E5F92402F5FB8005E5F904F5EA
:0618B400FBD21B22C21B47
:0118BA00220B
:03001E007F00223E
:10420D000218BBE493A3F8E493A34003F68001F2F4
:10421D0008DFF48029E493A3F85407240CC8C333B2
:10422D00C4540F4420C8834004F456800146F6DF81
:10423D00E4800B0102040810204080904B01E47EC5
:10424D00019360BCA3FF543F30E509541FFEE49376
:10425D00A360010ECF54C025E060A840B8E493A33D
:10426D00FAE493A3F8E493A3C8C582C8CAC583CA68
:10427D00F0A3C8C582C8CAC583CADFE9DEE780BE20
:014B070000AD
:102BAC00BB010CE58229F582E5833AF583E02250DE
:102BBC0006E92582F8E622BBFE06E92582F8E22228
:0D2BCC00E58229F582E5833AF583E4932242
:102BD900F8BB010DE58229F582E5833AF583E8F032
:102BE900225006E92582C8F622BBFE05E92582C8DE
:022BF900F222C6
:102BFB00E88FF0A4CC8BF0A42CFCE98EF0A42CFC79
:102C0B008AF0EDA42CFCEA8EF0A4CDA8F08BF0A4F6
:102C1B002DCC3825F0FDE98FF0A42CCD35F0FCEB55
:102C2B008EF0A4FEA9F0EB8FF0A4CFC5F02ECD391A
:0F2C3B00FEE43CFCEAA42DCE35F0FDE43CFC2287
:102C4A0075F008758200EF2FFFEE33FECD33CDCC41
:102C5A0033CCC58233C5829BED9AEC99E5829840C4
:102C6A000CF582EE9BFEED9AFDEC99FC0FD5F0D6A1
:102C7A00E4CEFBE4CDFAE4CCF9A88222B800C1B9CB
:102C8A000059BA002DEC8BF084CFCECDFCE5F0CB09
:102C9A00F97818EF2FFFEE33FEED33FDEC33FCEB42
:102CAA0033FB10D703994004EB99FB0FD8E5E4F9FD
:102CBA00FA227818EF2FFFEE33FEED33FDEC33FCEA
:102CCA00C933C910D7059BE99A4007EC9BFCE99ADE
:102CDA00F90FD8E0E4C9FAE4CCFB2275F010EF2F23
:102CEA00FFEE33FEED33FDCC33CCC833C810D70723
:102CFA009BEC9AE899400AED9BFDEC9AFCE899F85E
:0E2D0A000FD5F0DAE4CDFBE4CCFAE4C8F922F0
:0E2D1800C3E49FFFE49EFEE49DFDE49CFC22CC
:102D2600EB9FF5F0EA9E42F0E99D42F0E89C45F003
:012D3600227A
:102D3700E8600FECC313FCED13FDEE13FEEF13FF7A
:032D4700D8F1229E
:0C2D4A00ECF0A3EDF0A3EEF0A3EFF022FC
:102D5600A8828583F0D083D082122D6D122D6D123C
:102D66002D6D122D6DE473E493A3C583C5F0C58361
:102D7600C8C582C8F0A3C583C5F0C583C8C582C8C7
:012D8600222A
:102D8700D083D082F8E4937012740193700DA3A3DB
:102D970093F8740193F5828883E4737402936860EF
:062DA700EFA3A3A380DFEF
:10285000E569245DF8E6056922785A301702785D4B
:10286000E475F001122DD8022DAD2010EB7F2ED291
:10287000108018EF540F2490D43440D4FF30140B40
:10288000EF24BFB41A0050032461FFE56A6002150B
:102890006A056DE56D7002056C30170D785AE475A8
:1028A000F001122DD8EF022DC60248F47403D2179E
:1028B0008003E4C217F5698B5A8A5B895CE4F56A88
:1028C000F56CF56DE56A60077F2012288B80F57541
:1028D0006BFFC211C210C212C213C215C216C218B7
:1028E000122859FF700D3017057F0012289CAF6D1C
:1028F000AE6C22B4255FC2D5C214122859FF24D071
:10290000B40A00501A75F00A786A30D50508B6FF87
:102910000106C6A426F620D5047002D21380D9245D
:10292000CFB41A00EF5004C2E5D214022A9CD2118F
:1029300080C6D21080C0D21280BCD2D580BAD21547
:1029400080B47F2012288B2012077401B56A0040E2
:10295000F1122850FF12288B0228C4D218D21680F8
:1029600095122850FB122850FA122850F94A4B7041
:1029700006796D7A2B7BFF20122EE56A602A7E0095
:102980008E82758300122BAC60060EEE656B70F0C4
:10299000C2D5EBC0E0EAC0E0E9C0E0EE122AE3D025
:1029A000E0F9D0E0FAD0E0FB122DADFF60AAEBC059
:1029B000E0EAC0E0E9C0E012288BD0E02401F9D0C1
:1029C000E03400FAD0E0FBE56B0460DCD56BD98025
:1029D000877BFF7A2A79DFD212809C791080027976
:1029E00008C216C2188008D2D5790A8004790AC2B2
:1029F000D5E56B047002F56BE4FAFDFEFF1228507A
:102A0000FC7B08201113122850FD7B1030100A1295
:102A10002850FE122850FF7B20EC3382D592D550EF
:102A200013C3E43010069FFFE49EFEE42011039DD3
:102A3000FDE49CFCE4CBF8C211EC700CCFCECDCC05
:102A4000E824F8F870F38017C3EF33FFEE33FEEDA0
:102A500033FDEC33FCEB33FB994002FB0FD8E9EB81
:102A6000301105F8D0E0C448B211C0E00AEC4D4E78
:102A70004F78207B0070C2EAB56B0040BCC0E0120A
:102A80002AE5D0F0D0E0201104C4C0E0C4B211C0E7
:102A9000F0122874D0F0D5F0EB0228C4122D87294B
:102AA000615329DB5829324C292E4229DF4F29E76F
:0F2AB0004429E74929474329ED5529D14629D122
:102ABF004529D1472B8D5029362D293A2E295D2BAB
:102ACF00293E23295B202B762A28F648000029551A
:102ADF003F3F3F00790AA2D5201314301509B910D2
:102AEF00020404B9080104A2D520160250010420E3
:102AFF0012689212B56A005034C0E07F203013196B
:102B0F007F30A21272167215500F122B3CC212C2D6
:102B1F0016C215C2187F30800F301503E9C0E012BE
:102B2F00288B301503D0E0F9D0E0B56ACC301517FB
:102B3F007F30B9100C12288B7F583014077F7880A4
:102B4F0003B9080312288B3012057F2D02288B7FC3
:102B5F00202018F87F2B2016F322921280CF286E98
:102B6F00756C6C2900D2111228503011F8C21178EF
:102B7F006A30D50108F60228F62D5043495812281D
:102B8F00502403B405004001E4902B889312287C55
:0D2B9F00743A12287CD213756A040229DBF7
:10303B008B568A578958E4F562F561F560F55FF5B3
:10304B005DF55EE55A455B45596012EBC0E0EAC0A1
:10305B00E0E9C0E0AB59AA5AA95B122DE8AB5605C3
:10306B0058E558AA577002055714F9122DADF563A0
:10307B00C394094007E563D3940D40E1E5636420F5
:10308B0060DBE563B42D05435E038016E563B42B6B
:10309B0005435E01800C74FF2558F55874FF3557B6
:1030AB00F557E55C60046410703FAB56AA57A958FE
:1030BB00122DAD64306009E55C702E755C0A8029B9
:1030CB00900001122BACFF64786004EFB4581343EB
:1030DB005E01755C1074022558F558E43557F557A9
:1030EB008007E55C7003755C08AB560558E558AA7C
:1030FB00577002055714F9122DADF563C394614057
:10310B000AE563D3947A50035363DF74D02563F5D8
:10311B0063C3940A400CE5639411406D74F9256305
:10312B00F563E563D3955C5060435E01856267850B
:10313B006166856065855F64AF5C7E00E4FCFDAB1A
:10314B0062AA61A960A85F122BFBC8ECC8C9EDC9C4
:10315B00CAEECACBEFCBE4FCFDFEEB2563F562EECA
:10316B003AF561ED39F560EC38F55FAF62AE61AD04
:10317B0060FCAB67AA66A965A864D3122D26500321
:10318B000230F4435E040230F4E55E20E003E48099
:10319B002DE55A455B4559601EAB56E55824FFF9A2
:1031AB00E55734FFFAEBC0E0EAC0E0E9C0E0AB5909
:1031BB00AA5AA95B122DE8E55E30E20774FFFFFE09
:1031CB00FDFC22E55EAF62AE61AD60AC5F30E1034A
:0431DB00022D182287
:102DAD00BB010689828A83E0225002E722BBFE0224
:092DBD00E32289828A83E4932257
:102DC600BB010689828A83F0225002F722BBFE01EC
:022DD600F322E6
:102DD800FAE6FB0808E6F925F0F618E6CA3AF622FC
:102DE800BB011A89828A83D0F0D0E0F8D0E0F9D00C
:102DF800E0FAD0E0FBE8C0E0C0F0022E405016E94F
:102E0800F8D083D082D0E0F9D0E0FAD0E0FBC082DD
:102E1800C083022E37BBFE16E9F8D083D082D0E0FB
:0F2E2800F9D0E0FAD0E0FBC082C083022E49222D
:092E3700EBF608EAF608E9F622C0
:092E4000EBF0A3EAF0A3E9F02293
:092E4900EBF208EAF208E9F222BA
:00000001FF
